:020000040800F2
:1040000000C000203D7D0008997C00089B7C0008D2
:104010009D7C00089F7C0008A17C00080000000037
:10402000000000000000000000000000A37C000869
:10403000A57C000800000000A77C0008A97C0008FF
:10404000857D0008857D0008857D0008857D000848
:10405000857D0008857D0008AD7C0008857D000811
:10406000857D0008857D0008857D0008857D000828
:10407000857D0008857D0008857D0008B57C0008E9
:10408000C17C0008857D0008857D0008857D0008CD
:10409000857D0008857D0008857D0008857D0008F8
:1040A000857D0008857D0008857D0008857D0008E8
:1040B000857D0008857D0008857D0008857D0008D8
:1040C000857D0008857D0008857D0008857D0008C8
:1040D000857D0008CD7C0008D97C0008857D00081E
:1040E000857D0008857D0008857D0008857D0008A8
:1040F000857D0008857D0008857D0008857D000898
:10410000857D0008857D0008857D0008857D000887
:10411000857D0008857D0008E57C0008857D000818
:10412000857D0008857D0008857D0008857D000867
:10413000000000000000000000000000000000007F
:10414000000000000000000000000000000000006F
:10415000000000000000000000000000000000005F
:10416000000000000000000000000000000000004F
:10417000000000000000000000000000000000003F
:10418000000000000000000000000000000000002F
:10419000000000000000000000000000000000001F
:1041A000000000000000000000000000000000000F
:1041B00000000000000000000000000000000000FF
:1041C00000000000000000000000000000000000EF
:1041D00000000000000000000000000000000000DF
:0441E0005FF8E0F1B3
:1041E40010B5054C237833B9044B13B10448AFF32D
:1041F40000800123237010BD78000020000000001F
:10420400448F000808B5034B1BB103490348AFF3BF
:10421400008008BD000000007C000020448F0008DE
:1042240038B50E4B054618784FF47A73B3FBF0F3A8
:104234000B4A1068B0FBF3F000F09EF8044658B93E
:104244000F2D09D8024629464FF0FF3000F054F8EC
:10425400044B20461D6038BD012038BD00000020FD
:104264001000002004000020074A08B5136803204A
:1042740043F01003136000F02DF80020FFF7D0FF87
:1042840003F018FC002008BD00200240034A044B40
:1042940011681B780B441360704700BFB8050020F9
:1042A40000000020014B1868704700BFB8050020CB
:1042B40038B50446FFF7F6FF0546631C1EBF044BE2
:1042C4001B78E418FFF7EEFF401B8442FAD838BD90
:1042D40000000020074A0002D36800F4E06023F4E1
:1042E400E0631B041B0C43F0BF6343F4003303433C
:1042F400D360704700ED00E0174B30B5DC68C4F3C1
:104304000224C4F10703251D042B28BF0423062D12
:104314004FF0010598BF002405FA03F303F1FF33BE
:1043240088BF033C1940A14005FA04F4013C224033
:10433400002842EA01024FEA0212AFBF00F16040D6
:10434400064B00F00F00D2B2A5BFD2B200F5614017
:104354001A5480F8002330BD00ED00E014ED00E0B5
:104364000123420900F01F0003FA00F0014B43F857
:104374002200704700E100E00138B0F1807F0AD2EA
:10438400F021064B064A586082F8231000200722C9
:1043940098601A6070470120704700BF10E000E089
:1043A40000ED00E010B5002832D00168194B142448
:1043B400994225D8184AA3F207430A44B2FBF4F2FF
:1043C400920002648468C36343680A682343C46830
:1043D40022F47F522343046922F0300223434469C8
:1043E400234384692343C469234313430B60012299
:1043F400002380F82120836380F82030184610BD04
:10440400064B0B44B3FBF4F39B000364044BD9E762
:10441400012010BD07040240F8FFFDBFF8FBFDBFFB
:1044240000040240F0B590F82040012C35D001245E
:1044340090F8215080F82040A5424FF000064FF03C
:10444400020428D180F82140046886632668076C3A
:1044540026F001062660C66BBD4075606360436844
:104464000568102BC36A0BBFA260A160E160E26023
:104474004BB1236843F00E0323602B68002043F004
:1044840001032B60F0BD236823F004032360236839
:1044940043F00A03F0E780F820600220F0BD00003A
:1044A40090F8213010B5022B03D00423836301203C
:1044B40010BD03681A6822F00E021A601A6822F00E
:1044C40001021A60294A934224D902F56272934286
:1044D40019D01432934218D01432934217D01432A4
:1044E40093420CBF4FF480534FF48033204A5360FF
:1044F4000123002480F82130436B80F820409BB3D3
:104504009847204610BD0123F0E71023EEE74FF44F
:104514008073EBE717498B4216D014318B4215D0C8
:1045240014318B4214D014318B4214D014318B4289
:1045340014D014318B4214D0934214BF4FF48033FF
:104544004FF080730C4AD2E70123FBE71023F9E70D
:104554004FF48073F6E74FF48053F3E74FF480335E
:10456400F0E74FF48013EDE7184610BD80000240D9
:1045740000040240080002400000024070B4042518
:10458400C66B026C3468036895402542196855D09F
:104594004D0753D51A6896065EBF1A6822F00402C6
:1045A4001A60604A93421FD902F56272934214D092
:1045B4001432934213D01432934212D014329342E1
:1045C4000CBF4FF480434FF48023574A5360C36AAF
:1045D400002B00F0A58070BC18470423F5E74023A6
:1045E400F3E74FF48063F0E750498B4216D014315F
:1045F4008B4215D014318B4214D014318B4214D019
:1046040014318B4214D014318B4214D0934214BF12
:104614004FF480234FF08063454AD7E70423FBE738
:104624004023F9E74FF48063F6E74FF48043F3E760
:104634004FF48023F0E74FF48003EDE70225954023
:10464400254257D08D0755D51A68940606D41A68A2
:1046540022F00A021A60012280F82120314A934292
:104664001ED902F56272934213D01432934212D0CF
:104674001432934211D0143293420CBF4FF40053BE
:104684004FF40033284A5360002380F82030836AB3
:104694009EE70223F6E72023F4E74FF40073F1E7E3
:1046A40022498B4216D014318B4215D014318B42DF
:1046B40014D014318B4214D014318B4214D01431E1
:1046C4008B4214D0934214BF4FF400334FF0007365
:1046D400174AD8E70223FBE72023F9E74FF40073D6
:1046E400F6E74FF40053F3E74FF40033F0E74FF4E9
:1046F4000013EDE708259540254211D009070FD591
:10470400196821F00E011960012303FA02F27260A4
:10471400836380F82130002380F82030036B57E74F
:1047240070BC704780000240000402400800024050
:10473400000002402DE9F74F002216466C4F6D4BE6
:10474400DFF8B8E1DFF8B8C14FF001080C6808FAE7
:1047540006F808EA0404A04540F085804D68122D4F
:1047640000F0B78000F28D80022D00F0AF8000F2DF
:104774008180002D00F09180012D00F0A5804FF084
:104784000F09FF2C93BF824606F18045083DD0F8FF
:1047940000B092BFB500D0F804B0AD0009FA05F836
:1047A4002BEA080802FA05F588BF00F1040A48EA72
:1047B4000505CAF80050D1F804A01AF0805F52D061
:1047C400BD6926F0030845F00105BD61BD6908F126
:1047D400804805F00105019508F5803806F0030BC3
:1047E400019D4FEA8B0BD8F8085009FA0BF925EA1A
:1047F4000909414DA84271D005F58065A8426FD0E2
:1048040005F58065A8426DD005F58065A8426BD09A
:1048140005F58065A84269D070450CBF05250625BD
:1048240005FA0BF545EA0905C8F808501D681AF49D
:10483400803F14BF2543A5431D605D681AF4003F03
:1048440014BF2543A5435D609D681AF4801F14BFFF
:104854002543A5439D60DD681AF4001F14BF2C4353
:1048640025EA0404DC600136102E7FF46DAF03B03A
:10487400BDE8F08F032D25D0112D80D1CA680432F4
:104884007DE7654509D012D8DFF878904D4504D00E
:1048940009F580394D457FF472AF8A68E2B1012A87
:1048A4000CBFC0F81080C0F81480082267E7DFF856
:1048B40058904D45F1D009F580394D45EDD0A9F515
:1048C4008019E7E700225AE7CA6858E7CA6808323D
:1048D40055E7CA680C3252E7042250E700259FE7E7
:1048E40001259DE702259BE7032599E7042597E722
:1048F400001002400004014000080140001C014077
:1049040000002110000011100000311083681942CA
:1049140014BF0120002070470AB1016170470904E7
:10492400FBE7C3685940C1607047704708B5044B42
:104934005969014202D05861FFF7F7FF08BD00BF73
:10494400000401400268536913F480630DD06FF4CE
:10495400806353610423202203640023036380F8EB
:104964003C3080F83D2001207047184670472DE9FF
:10497400F843044617469946C1F307488EB22568A2
:10498400B8F1010F0CBF6B69AB6936EA030314BFBE
:104994000120002008B9BDE8F8836B695A0512D5D7
:1049A4002B68202243F400732B606FF480636B61E7
:1049B4000423236400230120236384F83C3084F817
:1049C4003D20BDE8F8837B1CD9D04FB900232022B9
:1049D400236384F83C3084F83D200320BDE8F88349
:1049E400FFF760FCA0EB09008742C8D2EEE72DE98F
:1049F400F843044690461F46089EC1F307498DB20A
:104A04002368B9F1010F0CBF5B699B6935EA0303A5
:104A14000CBF01230023434502D00020BDE8F883E6
:104A24007B1CEDD05FB900232022236384F83C3043
:104A340084F83D20032084F83E30BDE8F883FFF776
:104A440031FC801B8742DBD2EDE770B504460D468E
:104A5400164623685B691B0601D5002070BD2046FD
:104A6400FFF770FFA8B96A1CF3D065B9236C202244
:104A740043F02003236400230320236384F83C30A1
:104A840084F83D2070BDFFF70DFC801B8542E0D209
:104A9400ECE7012070BD00002DE9FF4115460268D6
:104AA400984613680B9E43F4807313600F46009678
:104AB4000A9B00224FF001110446FFF798FF68B9E2
:104AC400236807F0FE071F610A9A33461A492046F5
:104AD400FFF74DFF30B1236C042B18D0032004B032
:104AE400BDE8F081236803905A690A9903929B698F
:104AF400324603932046039BFFF7A7FF48B1236C7C
:104B0400042BEBD12268136843F400731360012073
:104B1400E5E7B8F1010F236802D1EDB21D61DEE7CC
:104B24002A0A1A610A9932462046FFF78EFF0028A6
:104B3400E5D12368F1E700BF020001002DE9FF4140
:104B44009846036816461A680B9D42F480621A6000
:104B54001A680F4642F480721A604FF001110095F2
:104B64000A9B00220446FFF742FF80B92368FFB284
:104B740007F0FE021A612D492B460A9A2046FFF7D8
:104B8400F6FE40B1236C042B01D1012000E0032088
:104B940004B0BDE8F081236803905A690A9903922E
:104BA4009B692A4603932046039BFFF74EFF40B1BF
:104BB400236C042BEBD12268136843F40073136055
:104BC400E3E7B8F1010F236824D1F6B21E612A4647
:104BD4000A992046FFF739FF02460028E8D12168E8
:104BE40020460B6843F480730B6000950A9B4FF0DA
:104BF4000111FFF7FCFE0028C9D1236847F0010723
:104C04001F610A9A2B4609492046FFF7B0FE002887
:104C1400B8D1BDE7320A1A610A992A462046FFF73D
:104C240014FF0028C4D12368CFE700BF02000100AD
:104C340070B504460D4616462068436913F04003D8
:104C440001D0002070BD4269D2060BD56FF010026E
:104C540042612022236484F83C302363012084F8D9
:104C64003D2070BD5DB9236C032043F02003236411
:104C7400202384F83D30002384F83C3070BDFFF7D6
:104C840011FB801B8542D7D2EDE770B504460D4673
:104C9400164623685B695B0701D5002070BD20467A
:104CA400FFF750FEA8B96A1CF3D065B9236C202223
:104CB40043F02003236400230320236384F83C305F
:104CC40084F83D2070BDFFF7EDFA801B8542E0D2E9
:104CD400ECE7012070BD000038B5044608B9012096
:104CE40038BD90F83D3003F0FF021BB980F83C203A
:104CF40002F002FF2423226884F83D30136823F075
:104D04000103136000F0BAFC63682F4A934230D861
:104D14002E4A9042E3D92E4A2168B0FBF2F24A604F
:104D240001320A62284A0138934232D85B00B0FB50
:104D3400F3F0431CC3F30B03042B38BF0423CB61F0
:104D4400226AE369002013430B60E268236913437A
:104D54008B60A26963691343CB600B6843F0010362
:104D64000B602023206484F83D30206384F83E00E7
:104D740038BD184A9042B2D9154D4FF49672B0FB23
:104D8400F5F521686A434D604FF47A75B2FBF5F28C
:104D9400C6E7A26852B903EB4303B0FBF3F0431C2C
:104DA400C3F30B036BB143F40043C8E71922534325
:104DB400B0FBF3F0431CC3F30B0313B143F44043C0
:104DC400BDE70123BBE700BFA08601007F841E006E
:104DD40040420F00FF083D002DE9F34704469A4680
:104DE400884691460C9EFFF75DFA94F83D300546DF
:104DF400202B03D0022002B0BDE8F08700901923D5
:104E040001223E492046FFF7F2FD0028F2D194F832
:104E14003C30012BEED0012384F83C30236800277A
:104E24001A684146D20758BF1A6820465CBF42F050
:104E340001021A601A6822F400621A60212384F8BD
:104E44003D30402384F83E300A9B27646362BDF8FA
:104E54002C30019563852A4B0096E362638D4A46A4
:104E640023855346FFF718FE00282AD0236C84F8C4
:104E74003C70042B07D10120BDE7FFF7E6FD20B10C
:104E8400236C042B34D00320B5E7616A27684B1CDC
:104E940063620B78228D3B61638D501E013B9BB294
:104EA40063857B6980B25B0720850AD548B18B1C7A
:104EB40063624B78023A3B61638D2285013B9BB26E
:104EC4006385238D2A4631462046002BD5D1FFF732
:104ED400DCFE0028D4D12268136843F40073136005
:104EE400202384F83C0084F83D3084F83E0082E7B7
:104EF4002268136843F400731360BCE702001000D7
:104F04000000FFFF2DE9F047044686B09A460D469F
:104F14009146109FFFF7C6F994F83D300646202BC2
:104F240004D00225284606B0BDE8F0870090192376
:104F3400012281492046FFF75AFD0028F1D194F857
:104F44003C30012BEDD0012384F83C3023684FF032
:104F540000081A682946D20758BF1A6820465CBF61
:104F640042F001021A601A6822F400621A602223D5
:104F740084F83D30402384F83E300E9BC4F84080D2
:104F84006362BDF83C30019663856C4B0097E36225
:104F9400638D4A4623855346FFF7D0FD054630B15D
:104FA400236C84F83C80042B3DD10125BAE7228D83
:104FB400236892B902905A6902929A690292029AFB
:104FC4001A6842F400721A60202384F83D300023EA
:104FD40084F83E3084F83C30A4E7012A25D11A68CD
:104FE40022F480621A6072B6236803905A690392AD
:104FF4009A690392039A1A6842F400721A6062B6BC
:10500400DFF83C81238D002BDED0032B77D8012BD6
:1050140027D1324639462046FFF70AFE00283FD002
:10502400236C202BC1D103257CE7022A1A680ED1F8
:1050340042F400621A6072B6236804905A690492BA
:105044009A690492049A1A6822F48062D6E742F4B8
:1050540080621A6005905A6905929B690593059BC5
:10506400CEE7022B00963B464FF000024146204615
:1050740024D1FFF7BCFC0028D5D172B623681A6886
:1050840042F400721A60626A1B69511C61621370F7
:10509400238D013B2385638D013B9BB2638562B6FF
:1050A400636A5A1C6262226812691A70238D013B7A
:1050B4002385638D013B9BB26385A3E7FFF797FCD0
:1050C40002460028AFD121680B6823F480630B608B
:1050D40072B6636A2046591C6162216809691970B5
:1050E400238D0096013B2385638D4146013B9BB292
:1050F40063853B46FFF77BFC0028BFD093E732462D
:1051040039462046FFF794FD002889D1636A5A1C6A
:105114006262226812691A70238D2268013B23851A
:10512400638D013B9BB2638553695B077FF56AAF6F
:10513400636A591C6162B7E7020010000000FFFFB8
:105144000400010038B50446D8B14CF6CC420368DB
:105154001A6045F255521A6042685A6082689A6031
:10516400FFF7A0F805462368D86818B94AF6AA22BA
:105174001A6038BDFFF796F8401B3028F3D9032096
:1051840038BD012038BD000003682DE9F341DB0779
:10519400054610D42B689F075ED42B68190700F1CD
:1051A40095802B685A0700F1BF80EA69002A40F015
:1051B4002D81002014E0904C636803F00C03042B51
:1051C40007D0636803F00C03082B0CD16368DE037B
:1051D40009D523689C03DDD56B68002BDAD1012047
:1051E40002B0BDE8F0816B68B3F5803F10D123684D
:1051F40043F480332360FFF755F806462368980389
:10520400C8D4FFF74FF8801B6428F7D90320E7E7D9
:105214009BB9236823F480332360236823F4802319
:105224002360FFF73FF8064623689903B2D5FFF7DA
:1052340039F8801B6428F7D9E8E7B3F5A02F236871
:1052440003D143F480232360D1E723F48033236024
:10525400236823F48023CDE7674C636813F00C0FB5
:1052640007D0636803F00C03082B10D16368DA03DA
:105274000DD423689B0702D52B69012BAFD123687A
:105284006A6923F0F80343EAC203236085E72A69C5
:105294005A4B6AB101221A60FFF704F806462368E4
:1052A4009F07ECD4FEF7FEFF801B0228F7D9ADE779
:1052B4001A60FEF7F7FF0646236898077FF56DAF7F
:1052C400FEF7F0FF801B0228F6D99FE7AA694A4C33
:1052D4004B4BDAB101221A60FEF7E4FF0646636A1B
:1052E4009B070DD54FF4FA52464B1B68B3FBF2F300
:1052F400019300BF019B5A1E0192002BF9D150E784
:10530400FEF7D0FF801B0228E9D97FE71A60FEF779
:10531400C9FF0646636A9F077FF543AFFEF7C2FFE6
:10532400801B0228F6D971E7334CE369D80024D4F2
:105334000127E36943F08053E361E36903F0805399
:105344000093009B304E3368D90518D5EB68012BC8
:1053540026D1236A43F001032362FEF7A3FF41F23F
:1053640088368046236A9B073FD5002F3FF41DAF44
:10537400E36923F08053E36117E70027E2E733682A
:1053840043F480733360FEF78DFF80463368DA059B
:10539400DCD4FEF787FFA0EB08006428F6D935E7D4
:1053A400ABB9236A41F2883823F001032362236AEC
:1053B40023F004032362FEF775FF0646236A980769
:1053C400D3D5FEF76FFF801B4045F7D91EE7052BA9
:1053D400236A03D143F004032362BAE723F00103F1
:1053E4002362236A23F00403B6E7FEF75BFFA0EB16
:1053F4000800B042B6D909E700100240000042425A
:10540400800442421000002000700040224C636877
:1054140003F00C03082B3FF4E2AE00231F4E022AD4
:1054240033602BD1FEF73EFF0746236899011FD452
:105434002B6AB3F5803F05D16268A96822F4003273
:105444000A436260696A62680B4322F4741213436C
:10545400636001233360FEF725FF054623689A0144
:105464003FF5A7AEFEF71EFF401B0228F6D9CDE696
:10547400FEF718FFC01B0228D7D9C7E6FEF712FFB4
:10548400054623689B017FF594AEFEF70BFF401B96
:105494000228F6D9BAE600BF00100240600042427A
:1054A40030B5194B87B002AC03F1100522461868D9
:1054B4005968083303C2AB421446F7D101238DF86F
:1054C4000430022311498DF805304B6803F00C02B7
:1054D400082A17D1C3F3834206A80244DB0312F857
:1054E400102C0CD54B680A48C3F34043504306AA1A
:1054F400134413F8143CB0FBF3F007B030BD054877
:105504005043FAE70248F8E75C8F000800100240B5
:1055140000127A0000093D00544A2DE9F041136855
:10552400054603F007038B420E462AD329688C07ED
:1055340034D4CA0747D44D4A136803F007039E4284
:10554400C0F082802A684A4C12F0040F40F0878031
:10555400130706D563682A6923F4605343EAC20338
:105564006360FFF79DFF6368424AC3F30313D35C90
:10557400D840414B18600020FEF752FE0020BDE8E1
:10558400F081136823F007030B431360136803F0DF
:1055940007039942CAD00120BDE8F081344B11F0D1
:1055A400040F1EBF5A6842F4E0625A60080742BF03
:1055B4005A6842F460525A605A68A86822F0F002AD
:1055C40002435A60B5E76A68294C012A23681CD152
:1055D40013F4003FDFD0636841F2883823F00303FB
:1055E40013436360FEF75EFE6B680746012B14D11C
:1055F400636803F00C03042B9DD0FEF753FEC01B1D
:105604004045F5D90320BDE8F081022A02D113F008
:10561400007FDFE713F0020FDCE7022B0FD1636892
:1056240003F00C03082B86D0FEF73CFEC01B40455C
:10563400F5D9E7E7FEF736FEC01B4045E2D86368BC
:1056440013F00C0FF6D176E7136823F00703334306
:105654001360136803F007039E429CD172E76368EA
:10566400E96823F4E0630B43636071E700200240C0
:10567400001002406791000810000020044B054A06
:105684005B68C3F30223D35C034A1068D8407047B5
:10569400001002407791000810000020044B054AD6
:1056A4005B68C3F3C223D35C034A1068D8407047D5
:1056B40000100240779100081000002003680020C9
:1056C400DA6842F00102DA601A6842F001021A60F4
:1056D40070477047704770477047036810B51A6980
:1056E400044691070ED5DA6892070BD56FF00202D3
:1056F4001A6101229B6902779B0777D0FFF7EAFFC3
:105704000023237723681A69500710D5DA685107F4
:105714000DD56FF004021A6102229B69227713F4FB
:10572400407F204668D0FFF7D5FF00232377236806
:105734001A6912070FD5DA6810070CD56FF0080242
:105744001A610422DB692277990720465AD0FFF7B1
:10575400C1FF0023237723681A69D20610D5DA68BB
:10576400D0060DD56FF010021A610822DB6922778A
:1057740013F4407F20464BD0FFF7ACFF0023237780
:1057840023681A69D10708D5DA68D20705D56FF0FE
:10579400010220461A6101F039FC23681A691006D7
:1057A40008D5DA68110605D56FF0800220461A6123
:1057B40000F0BFF823681A69520608D5DA68500663
:1057C40005D56FF0400220461A61FFF785FF236874
:1057D4001A69910622D5DA6892061FD56FF0200265
:1057E4002046BDE810401A6100F0A2B8FFF771FF2F
:1057F4002046FFF770FF83E7FFF76BFF2046FFF7B4
:105804006AFF92E7FFF765FF2046FFF764FFA0E712
:10581400FFF75FFF2046FFF75EFFAFE710BD000014
:10582400244A0368904212D002F5006290420ED0DE
:10583400B0F1804F0BD0A2F59832904207D002F518
:105844008062904203D002F5806290421DD14A6882
:1058540023F070031343174A904212D002F50062FA
:1058640090420ED0B0F1804F0BD0A2F59832904206
:1058740007D002F58062904203D002F58062904224
:1058840003D1CA6823F4407313434A6923F08003A5
:10589400134303608B68C3620B688362054B9842B1
:1058A40003D003F50063984201D10B69036301231C
:1058B40043617047002C014010B50446A0B190F834
:1058C4003D3003F0FF021BB980F83C2002F046F99A
:1058D4000223206884F83D30211DFFF7A1FF012336
:1058E400002084F83D3010BD012010BD90F83C30FC
:1058F40010B5012B4FF0020318D080F83D30036837
:105904000C685A68496822F070025A605A68224347
:105914005A609A6822F080029A609A680A439A60F0
:10592400012380F83D30002380F83C30184610BD38
:10593400704770470368DA6822F49072DA605A6933
:1059440022F001025A61202380F83A3070470000A7
:105954002DE9F0470568C2682B69016923F44053B7
:1059640013432B618368EA680B43416922F4B05204
:1059740022F00C020B431343EB606B69826923F43E
:10598400407313436B61404B81469D424FF01904B1
:1059940046D1FFF783FE04FB00F3D9F804604FF00F
:1059A4006408B600B3FBF6F3B3FBF8F31E01FFF78C
:1059B40075FE6043D9F804309B00B0FBF3F7FFF7A2
:1059C4006DFE6043D9F804309B00B0FBF3F3B3FBE6
:1059D400F8F308FB13731B013233B3FBF8F303F042
:1059E400F007FFF75BFE6043D9F804209200B0FB98
:1059F400F2FAFFF753FE6043D9F804309B00B0FB82
:105A0400F3F3B3FBF8F308FB13A31B013233B3FB2B
:105A1400F8F303F00F033B433344AB60BDE8F08776
:105A2400FFF72CFE04FB00F3D9F804604FF0640880
:105A3400B600B3FBF6F3B3FBF8F31E01FFF71EFE4B
:105A44006043D9F804309B00B0FBF3F7FFF716FE70
:105A54006043D9F804309B00B0FBF3F3B3FBF8F3D5
:105A640008FB13731B013233B3FBF8F303F0F007A5
:105A7400FFF704FE6043D9F804209200B0FBF2FA69
:105A8400FFF7FCFDB7E700BF00380140F8B5044656
:105A94000E4617461D4621680B6836EA030301D1FA
:105AA4000020F8BD6B1CF7D095B923680320DA6891
:105AB40022F4D072DA605A6922F001025A6120237A
:105AC40084F8393084F83A30002384F83830F8BD4B
:105AD400FEF7E8FBC01B8542DDD2E6E710B50446BD
:105AE40040B390F8393003F0FF021BB980F8382036
:105AF40002F048F82423226884F83930D368204619
:105B040023F40053D360FFF723FF236800201A69AE
:105B140022F490421A615A6922F02A025A61DA6820
:105B240042F40052DA602023E06384F8393084F8C8
:105B34003A3010BD012010BD2DE9F0411F4690F808
:105B440039300446202B0D4690464ED1002949D0C9
:105B5400002A47D090F83830012B46D0012380F832
:105B640038300023C363212380F83930FEF79AFBD1
:105B74000646A4F82480A4F82680E38C9BB26BB973
:105B84003B46324640212046FFF780FFA8B9202338
:105B940084F8380084F83930BDE8F081E38C32466B
:105BA400013B9BB2E384A3688021B3F5805F204668
:105BB4003B460ED1FFF76AFF10B10320BDE8F08128
:105BC4002B882268C3F308035360236943B9023561
:105BD400D3E7FFF75BFF0028EFD123682A785A60E8
:105BE4000135CAE70120BDE8F0810220BDE8F0815B
:105BF400134690F83A2073B5202A054638D1002977
:105C040034D0002B32D090F83820012A30D0012231
:105C1400002480F83820222281628385C46380F8BE
:105C24003A20406B134A2E688262134A4463C2626C
:105C3400124A02630A46311DFEF7F4FB20462B6824
:105C440001941A6801925A6885F838400192019AC1
:105C5400DA6842F48072DA605A6942F001025A61E9
:105C64005A6942F040025A6102B070BD0120FBE75C
:105C74000220F9E7875C00083D5D0008495D0008E3
:105C8400704708B50368426A1B6813F0200310D1FB
:105C9400D3851368D96821F48071D960596921F0DA
:105CA40001015961596921F040015961202382F8A9
:105CB4003A30104601F078F908BD90F83A3010B542
:105CC400222B36D183680169B3F5805F0268836A49
:105CD40023D15268E9B9C2F3080223F8022B836284
:105CE400C48D013CA4B2C4858CB90368DA6822F07F
:105CF4002002DA60DA6822F48072DA605A6922F0EB
:105D040001025A61202380F83A3001F04DF9002055
:105D140010BDD2B223F8012BE1E721B9591C526816
:105D240081621A70DCE75268591C816202F07F02BA
:105D3400F7E7022010BD704708B5406AFFF7FBFF84
:105D440008BD7047416A08B50B685A6991F8390073
:105D540021280AD1120608D50022CA84DA6822F062
:105D6400C002DA60202281F839205B6991F83A2078
:105D7400222A06D15B0604D500230846CB85FFF70B
:105D8400D9FDCB6B084643F01003CB63FFF7D9FF73
:105D940008BD0000036870B51A6804461607D96880
:105DA4005D6907D196065AD58D0658D5BDE8704071
:105DB400FFF783BF15F0010502D111F4907F4ED097
:105DC400D30705D5CE0542BFE36B43F00103E3637C
:105DD400500704D51DB1E36B43F00203E36393075B
:105DE40004D51DB1E36B43F00403E363160704D544
:105DF4001DB1E36B43F00803E363E36B002B66D050
:105E0400950604D5880602D52046FFF756FF236879
:105E140020465D69E26B110702D415F040051AD0E3
:105E2400FFF788FD23685A69520610D55A69606BDA
:105E340022F040025A6150B1254B4363FEF730FB18
:105E4400002844D0606BBDE87040436B184720467F
:105E5400FFF777FF70BDFFF774FFE56370BD1606AB
:105E640027D50D0625D594F83920212A2FD1A268EB
:105E7400B2F5805F226A17D11188C1F30801596015
:105E8400216979B902322262E28C013A92B2E28447
:105E9400EAB9DA6822F08002DA60DA6842F0400295
:105EA400DA6070BD0132EEE7511C216212785A604B
:105EB400EAE750060BD54A0609D5DA68204622F0EF
:105EC4004002DA60202384F83930FFF7D9FE70BD30
:105ED400D95E000808B50023406AC385C384FFF770
:105EE40030FF08BD002382B00093009B834201DB96
:105EF40002B07047019B01330193009B0133F3E728
:105F040070B505460824144E0420FFF7EBFF002269
:105F140008213046FEF700FD2B064CBF012200226B
:105F240020213046FEF7F8FC0420FFF7DBFF0122B6
:105F340008213046FEF7F0FC013C04206D00FFF719
:105F4400D1FF14F0FF04EDB2DED12246BDE870406B
:105F540008210148FEF7E0BC000C014070B508259B
:105F64000024104E0420FFF7BDFF08213046012213
:105F7400FEF7D2FC640010213046E4B2FEF7C6FC02
:105F840008B144F001040420FFF7ACFF013D0022F6
:105F940008213046FEF7C0FC15F0FF05E2D120468B
:105FA40070BD00BF000C0140FFF7AABF2DE9F04F00
:105FB40006460F4690461D4600244FF4FA694FF0FA
:105FC400010ADFF840B087B0AC4202D107B0BDE8A7
:105FD400F08F3B1908EB0402009392B21023A02126
:105FE400CDF80890CDF804A03046FEF7F5FE0590F4
:105FF4000520FEF75DF9059B13B1584601F082FFB9
:106004000134E1E76C8F00087FB5002206AB03F88A
:10601400042D4FF4FA62029201220093019210239C
:106024000A46A121FEF76EFF9DF8140007B05DF843
:1060340004FB00000138C0B207289ABF014B185C6A
:1060440000207047828F00080138C0B207289ABF29
:10605400024B33F810000020704700BF8A8F0008FD
:106064002DE9F74F00216848684EFFF7CDFF012462
:10607400B046674D644F287021463846FFF7C4FF89
:10608400611C0002708089B23846FFF7BDFF0634F8
:106094007388A4B21843312C26F8020FECD1DFF830
:1060A4009C9103244F46584E21463046FFF7ACFFDF
:1060B400611C0002A9F8020089B23046FFF7A4FF70
:1060C4000634B9F80230A4B21843332C29F8020F6D
:1060D400EAD1DFF86C910524CB464B4E214630467D
:1060E400FFF792FF611C0002A9F8020089B2304652
:1060F400FFF78AFF0634B9F80230A4B21843352CEE
:1061040029F8020FEAD100244FF03209661CF0B2DC
:10611400FFF79AFF4FF0000A024609FB04F402EB72
:106124000A0189B238480192FFF76EFF394B0AEB36
:1061340004010AF1010A1944BAF1320F81F832005C
:10614400019AECD1082E3446E0D12978324801F086
:1061540051FE0124DFF8EC90304E314D38F8142014
:106164002146484601F046FE37F8142021463046C1
:1061740001F040FE3BF8142021462846013401F08A
:1061840039FE092CEAD14FF4E1711F48FFF73CFFB7
:10619400FF2835D04FF4E1711B48FFF735FF214C40
:1061A40040F2C31120701848FFF72EFF4FF4E2713C
:1061B40060701548FFF728FF40F2C511A07012481F
:1061C400FFF722FF4FF4E371E0700F48FFF71CFF65
:1061D40021782071144801F00DFE6178134801F014
:1061E40009FEA178124801F005FEE178114801F09A
:1061F40001FE2179104803B0BDE8F04F01F0FABD6B
:1062040003B0BDE8F08F00BF140600209C030020FB
:106214000804002002010020B78F0008EC8F00085A
:1062240013900008080000203A90000850900008DD
:10623400669000087C900008929000088A03002071
:10624400C4020020C58F00082DE9F34143780446B9
:10625400013B1A2B00F2A380DFE803F0330E33A1D5
:106264001A2733333AA1A1A1A13E4765A165A1A193
:10627400A1768865A1A165000A2100F001FF012330
:1062840000224849484802B0BDE8F041FFF78EBEFD
:10629400A27821461424C078444B033204FB003016
:1062A40002B0BDE8F04101F091BD81780331C9B27B
:1062B40000F0E6FEA07AFFF7BDFE06230246211D8C
:1062C400E0E70721204602B0BDE8F04100F0D0BE6F
:1062D40081780331C9B2F5E7C078FFF7B5FEA3783A
:1062E40002460333DBB22146CCE7807AFFF7ACFEEB
:1062F400811C89B22C48FFF787FEA070E078FFF775
:10630400A3FE00230746DFF8A080A178DEB25D1C5F
:106314008B1CB34210DA20460F2300F8013F4D1CBA
:1063240001F08FFB60552046A1780331C9B202B059
:10633400BDE8F04100F0A4BEB91989B24046FFF7A8
:1063440063FE2B46A055E0E7827801460332684697
:1063540001F03CFD134B9DF804201B789A421ED19A
:10636400012002B0BDE8F04100F076BE1823C278E7
:1063740043700F4B1A7002795A7142799A7082797C
:10638400DA70C2791A7100F0D3FFA3784FF4E17286
:10639400023BDBB2E11C0448FFF708FEC3E702B08E
:1063A400BDE8F0810804002014060020D602002075
:1063B4000800002008B5082850D8DFE800F00530B0
:1063C400383C4044484B2C0000224FF48061244860
:1063D400FEF7A2FA00224FF400612148FEF79CFA6E
:1063E40000224FF480511E48FEF796FA0022042141
:1063F4001C48FEF791FA002240211B48FEF78CFA54
:10640400002280211848FEF787FA00224FF4807199
:106414001548FEF781FA00224FF4007115E00022BE
:106424004FF480610E48BDE80840FEF775BA0022BB
:106434004FF40061F6E700224FF48051F2E70022A6
:1064440004210848EFE7002240210748EBE7002237
:106454008021FAE700224FF48071F6E708BD00BFFF
:106464000010014000140140000C014008B5082848
:1064740050D8DFE800F00530383C4044484B2C004D
:1064840001224FF480612448FEF746FA01224FF4BA
:1064940000612148FEF740FA01224FF480511E4862
:1064A400FEF73AFA012204211C48FEF735FA0122CC
:1064B40040211B48FEF730FA012280211848FEF7DC
:1064C4002BFA01224FF480711548FEF725FA0122B8
:1064D4004FF4007115E001224FF480610E48BDE8CD
:1064E4000840FEF719BA01224FF40061F6E70122D1
:1064F4004FF48051F2E7012204210848EFE701221A
:1065040040210748EBE701228021FAE701224FF4FA
:106514008071F6E708BD00BF00100140001401407F
:10652400000C01402DE9F04700252C46DFF860906F
:10653400DFF86080DFF860A099F80030EFB2BB426A
:106544000BD20CBB224611484FF48051FEF7E4F9FC
:106554002046BDE8F047FFF789BF18F807001AF88E
:106564000060012E0CD1094832464FF48051FEF7E9
:10657400D3F918F80700FFF71DFF01353446DBE7B0
:10658400FFF774FF2646F8E7BDE8F087000C0140EA
:10659400AE030020AF03002094000020002230B599
:1065A40010460125074B084C1978D3B2994200D8FC
:1065B40030BD135D23B1013B05FA03F31843C0B2A8
:1065C4000132F2E7AE030020AF0300200138C0B26D
:1065D40007289ABF014B185C002070479A8F000867
:1065E400F8B5BE231D4C00222370EB236260E371D7
:1065F400162363700523A370194B1A4E1B780546A6
:106604003078E370FFF7E2FFC8B1174B4FF0010E8B
:106614001F7813462179D8B2B84215D902B1217135
:106624000023EA5C61799A4001330A43082B6271C2
:10663400F7D105210D4801F004FAA071F8BD0C480A
:10664400BDE8F84001F05EBC325C0133013A0EFA59
:1066540002F21143C9B20122DDE700BF9D00002010
:1066640008040020AF030020AE0300209E00002099
:10667400A89000082DE9F74F8179C279C378264E96
:1066840042EA0122047A26F81320427A234942EA94
:10669400042221F81320847AC27A214D42EA04228A
:1066A40025F8132000224FF0010E144691461D4B8D
:1066B400284693F800C01C4F1C4DDFF884800191DC
:1066C400D3B263450AD91A48FFF78AFF194B1A78DF
:1066D400A24218BF1C7003B0BDE8F08F1649CB5C12
:1066E40037F813B036F813A0D3450DD8134931F851
:1066F40013B0019931F813A0D34505D838F813B075
:1067040030F813A0D34504D9012405F803E001327D
:10671400D6E705F80390FAE7DC030020CA0300205B
:10672400B8030020AE0300209C0300209400002046
:106734009500002001010020AF0300208A030020FF
:10674400C402002030B545789BB004466422002181
:1067540001A801F046FB6B1E1A2B38D8DFE813F0B2
:106764001B003C00460058006600980037003700C4
:106774003700BF00370037003700CC00D300DA0001
:106784003700F10037003700200137002A013C01AF
:10679400370037005F01B44AB44811784B1C415CA0
:1067A400DBB22171B24913700978601C994238BF79
:1067B4000023A17838BF137001F043F96071A288F7
:1067C4002068A3790190ADF808208DF80A3001A85B
:1067D400FFF73AFD1BB030BDA2782146033201A871
:1067E40001F0F4FAE278A34B1A70F0E7012000F00C
:1067F40039FCA2782146033201A801F0E7FA9DF89A
:1068040006100DF1050001F01CF98DF80900DEE712
:10681400E1780029DED0984801F0ECFA944A137824
:10682400591C1170E178914AD154D0E70021E378E2
:10683400924A2046D154A3780133A370FFF71AFF7C
:10684400A2782146033201A801F0C0FAFFF7A6FEA0
:106854009DF806301AAA134403F8650C9DF8063017
:106864000DF105001344864A527903F8642C9DF80F
:106874000640214601F0E5F81AAB1C4404F8630C09
:106884009DF806301AAA1344EB2203F8622C9EE703
:10689400A2782146033201A801F098FA227963799B
:1068A400A17A43EA0223774A0DF1050022F8113058
:1068B400A279E379A17A43EA0223734A22F81130D8
:1068C400227A637AA17A43EA0223704A22F81130C9
:1068D4009DF8061001F0B5F88DF80F0077E7BFF3C7
:1068E4004F8F6B496B4BCA6802F4E0621343CB6071
:1068F400BFF34F8F00BFFDE7A2782146033201A802
:1069040001F064FA63E70F238DF80530E3788DF81E
:1069140007305CE7BE238DF80430102303218DF883
:106924000530544B0DF105001B788DF806108DF8D9
:10693400073001F086F8EB238DF808008DF8093054
:1069440045E7BE238DF80430122308218DF8053065
:106954004C4AE3788DF8061032F8132022FA01F03D
:106964008DF80820484A8DF8070032F8132022FADF
:1069740001F08DF80A20454A8DF8090032F81330E9
:106984000DF1050023FA01F28DF80C308DF80B207F
:1069940001F057F8EB238DF80D008DF80E3016E753
:1069A400A2782146033201A801F010FA16238DF8CB
:1069B40005300CE7384800F0BCF8A57821460335CB
:1069C4002A4601A801F002FA9DF806100DF105000F
:1069D40001F037F86055FAE6BE238DF8043012232F
:1069E40007218DF805302D4B0DF105001A798DF82E
:1069F40006108DF807205A7A8DF80820DA798DF878
:106A040009209A791B7A8DF80A208DF80B3001F051
:106A140018F8EB238DF80C008DF80D30D7E6204DD7
:106A2400124A2B7801A8D15C14225C1C1D4BE4B2E1
:106A340002FB01318A782C70033201F0C7F90C4B48
:106A44000DF105001B78A3423CBF00232B701B23D0
:106A54009DF806408DF80530214600F0F2FF1AAB90
:106A64001C4404F8630CB2E6F8030020AF030020D2
:106A7400AE03002008040020A28F0008EE030020CB
:106A84009D0000209C0300208A030020C4020020F3
:106A940000ED00E00400FA05D006002024090020DF
:106AA400F7030020D60200204B1E5A42018A5A41A5
:106AB4004069FDF731BF10B504460121FFF7F4FF2B
:106AC400218860680122BDE81040FDF725BF10B59C
:106AD4000C460021FFF7E8FF2046BDE81040FFF711
:106AE40063BAF8B50E4604461F46002100681546F1
:106AF400FFF7DAFF46F080012068FFF7E8FF013F67
:106B04006E1E3D44AE4204D101212068FFF7CCFF44
:106B1400F8BD16F8011F2068FFF7D9FFF2E708B5A2
:106B24000021FFF7C1FFFFF719FAC0B208BDFDF756
:106B3400BFBB10B504460121FFF7B6FF2188002230
:106B44006068FDF7E9FE0120FFF7F1FF60680122AC
:106B54002188FDF7E1FE6420FFF7E9FF10BD08B5C9
:106B64000189C068FDF7D2FE431E5842584108BD52
:106B740038B504460068FFF7AAFF2068FFF7CFFF87
:106B8400054601212068FFF78FFF284638BD70B500
:106B940004460E46154600210068FFF785FF46F0BF
:106BA40080012068FFF793FF29462068FFF78FFFD5
:106BB40001212068FFF778FF70BD012BF8B5054669
:106BC4000F4616461C4616D900210068FFF76CFFD5
:106BD40039462868FFF77BFF013CE4B2771E344452
:106BE4002868FFF79CFF07F8010FA742F8D101219D
:106BF4002868FFF759FFF8BD012B01D9FFF771BFD2
:106C040070474279437A02F00F0242F0700242EA7E
:106C1400C312D2B20921FFF7BABF10B5092201216C
:106C24000446FFF7B4FF0123E37210BD10B5082238
:106C340001210446FFF7ABFF0023E37210BD882255
:106C44000121FFF7A4BF00002DE9F84304460D46D7
:106C540091461F469DF820609DF82480FFF7E6FFCB
:106C64000F20FFF764FF2046FFF7E9FF344A05EBE6
:106C740045052A44032306212046FFF732FF314B02
:106C8400092113F809202046FFF781FF0B22204633
:106C94001146FFF77CFF2046FFF7B3FF42460C2165
:106CA4002046FFF774FF284BDD5D284B062D9A5DC7
:106CB4004FEA021237D10332D2B21D212046FFF728
:106CC40066FF67221E212046FFF761FF312120461F
:106CD400FFF74EFF00F0F80242F005023121204692
:106CE400FFF755FF0C2237212046FFF750FF2046BF
:106CF400FF221F21FFF74BFF204600222021FFF730
:106D040046FF20460C222121FFF741FF20460122A5
:106D14004121FFF73CFF0023204684F80C31BDE8F5
:106D2400F843FFF77ABF023202F0FE021D2120462B
:106D3400FFF72DFF2A010732D2B21E21D4E700BF8C
:106D4400BA900008EE900008F2900008E490000861
:106D540030B5457A85B00295C479057A837942794C
:106D6400017901950094FFF76FFF05B030BDFF2254
:106D74001221FFF70CBF70B504460E46A1721546EA
:106D8400FFF7E6FF84224D212046FFF700FFFF2294
:106D940024212046FFF7FBFE012240212046FFF775
:106DA400F6FE3F2211212046FFF7F1FE2046FFF7B1
:106DB400DEFF324622212046FFF7E9FE0F2120465E
:106DC400FFF7D6FE0D2102462046FFF7E0FE85229E
:106DD40001212046FFF7DBFE002384F80C31182143
:106DE4002046FFF7C5FE430703D503230120E372C2
:106DF40070BD013D07D12068FFF79BFE2046FFF7D9
:106E0400A7FF284670BD0120FFF791FEE7E770B5A4
:106E140004460068FFF7A3FEF0B104F10C064FF43A
:106E240080720021304600F0DCFF10212046FFF77D
:106E34009FFE0D2102462046FFF7A9FEA37973B9F0
:106E4400A57A20462B4632460021FFF7B6FE84F889
:106E54000C512046FFF78BFF94F80C0170BD1321F1
:106E64002046FFF785FE0546EBE770B504460E465F
:106E7400A1721546FFF76CFF87224D212046FFF7CC
:106E840086FE002224212046FFF781FE4122402174
:106E94002046FFF77CFE2046FFF769FFF722112109
:106EA4002046FFF774FE324622212046FFF76FFE8C
:106EB4000E212046FFF75CFE0D2102462046FFF717
:106EC40066FE22212046FFF753FE864203D10223A9
:106ED4000120E37270BD013DF3D12068FFF729FE64
:106EE4002046FFF735FF284670BD70B504461E46A0
:106EF40013460A460021FFF77FFE8B22012120461C
:106F0400FFF745FE2068FFF72AFE054660B112210F
:106F14002046FFF72DFE2046FFF729FF2046FFF706
:106F24007CFE0125284670BD013E06D12068FFF78E
:106F340000FE2046FFF70CFFF4E70120FFF7F7FD02
:106F4400E0E72DE9F84F04468B46924699469DF8B2
:106F540028809DF82C709DF830609DF834500068AE
:106F6400FFF7A9FD84F804B084F805A084F806901E
:106F740084F80780A772267265722046BDE8F84F30
:106F8400FFF7E6BE70B50E4690F80C41054600F1D9
:106F94000C012246304600F019FF0023335585F8D2
:106FA4000C31204670BD00000268104B10B59A42A7
:106FB4000BD10F4A0F4913780C780F49CC54013385
:106FC400DBB2632B88BF0023137002680B4B9A4219
:106FD4000BD10B4A0B49137808780B49C854013379
:106FE400DBB2632B88BF0023137010BD003801404F
:106FF400DE0400203C08002014040020004400406B
:10700400DF040020680600207804002002680C4B8E
:107014009A4213D10B4A1368013313600A4A136866
:1070240001331360094A136801331360084A136873
:1070340001331360074A136801331360704700BFBC
:10704400001000400C04002010040020FC03002069
:107054000404002000040020014B1870704700BF96
:10706400EC060020014B1870704700BF0904002093
:107074000A460A2301460148FEF75EBDE0080020E7
:107084000A460A2301460148FEF756BD340700208C
:1070940010B514460A230248FEF74EFD204610BDE3
:1070A40034070020F8B50D468178044643185A7811
:1070B400013000F0E1FCC8B9114F2B78461CC0B276
:1070C40083420DD8A378002123445A780D4800F058
:1070D40091FE2046BDE8F8406422002100F081BE04
:1070E400215C384600F086FE3046E6E7012803D1ED
:1070F4002046FFF727FBECE7034800F003FFE8E72F
:10710400179100081D91000843910008BE2313B590
:1071140002218DF80030192304460DF101008DF889
:1071240001308DF8021000F08CFCEB238DF8030085
:107134008DF80430082C44D8DFE804F0CA05454D26
:107144005B6F88A6CA009DF8021068460331C9B275
:10715400FFF796FF00224FF400517248FDF7DCFB65
:107164006420FDF7A5F801224FF400516D48FDF7A6
:10717400D3FB00224FF480416A48FDF7CDFB002287
:107184004FF400416748FDF7C7FB002240216648E1
:10719400FDF7C2FB002280216348FDF7BDFB0022FE
:1071A4004FF480716048FDF7B7FB00224FF4007183
:1071B4005D48FDF7B1FB00224FF480715B48FDF799
:1071C400ABFB02B010BD01224FF400515548FDF74E
:1071D400A3FB0122CEE701224FF400515148FDF7F1
:1071E4009BFB01224FF480414E48FDF795FB0122A1
:1071F400C6E701224FF400514A48FDF78DFB0122F6
:107204004FF480414748FDF787FB01224FF40041CA
:107214004448FDF781FB0122B8E701224FF40051F5
:107224004048FDF779FB01224FF480413D48FDF7CA
:1072340073FB01224FF400413A48FDF76DFB012234
:1072440040213948FDF768FB0122A4E701224FF4ED
:1072540000513448FDF760FB01224FF4804131486E
:10726400FDF75AFB01224FF400412E48FDF754FB71
:10727400012240212C48FDF74FFB012280212A489E
:10728400FDF74AFB01228BE701224FF40051254808
:10729400FDF742FB01224FF480412248FDF73CFBFD
:1072A40001224FF400411F48FDF736FB0122402123
:1072B4001D48FDF731FB012280211B48FDF72CFB03
:1072C40001224FF480711848FDF726FB01226DE777
:1072D40001224FF400511348FDF71EFB01224FF425
:1072E40080411048FDF718FB01224FF400410D487E
:1072F400FDF712FB012240210B48FDF70DFB012293
:1073040080210948FDF708FB01224FF480710648EB
:10731400FDF702FB01224FF400710348FDF7FCFA6C
:10732400012249E7000C014000100140000801401F
:107334001021164B164A30B5DA605A614FF40042F8
:107344009960012113481A614579134C134A85B099
:1073540083E80600236042788378017803950579F1
:1073640002950A250195C07800902046FFF7E9FDB3
:1073740000220B4B08211A6020464FF4FA62FFF7F3
:10738400FAFC084B186005B030BD00BFD0060020E1
:10739400000801400800002024090020000C0140DE
:1073A400340A0020200900202DE9F0412E4E2F4DF3
:1073B4003378012B31D108212D4A2E4C13682E4FDE
:1073C400236053682D4863604FF4FA623960FFF715
:1073D4004CFD3A7828604FF4FA6321462748FFF7BA
:1073E40084FD2860264800F005FD0027DFF898801A
:1073F400E15D4046013700F0FDFC072FF8D10A207B
:1074040000F010FD00234FF4FA6208211B4833708A
:10741400FFF7B1FC2860BDE8F0811848FFF7F7FCDE
:1074240002462860E8B113491448FFF7ABFD15483C
:1074340000F0E0FC00240F4E134F2A68E3B293429D
:1074440004F1010408DB0A2000F0ECFCBDE8F04183
:1074540006490848FFF726BEF15C384600F0CAFC2E
:10746400EBE7BDE8F08100BFEC0600202009002016
:107474009D0000207407002000060020240900203D
:10748400F9900008069100081791000870B5314A78
:10749400314B11781B78314C8B4213D0304B187818
:1074A400451C1D704B1CDBB21370632B4FF00003A3
:1074B40088BF13702B4A2C4D136001236D5C2B493C
:1074C40023700D542A4A2B4B11781B788B4213D00E
:1074D400294B1878451C1D704B1CDBB21370632BB1
:1074E4004FF0000388BF1370244A254D1360022314
:1074F4006D5C244923700D542278234D012A2A708F
:1075040010D1184B1B68642B0CD90026144B12495C
:1075140016481E702670FFF7C5FD642231461348D5
:1075240000F05FFC2B78022B12D1144B1B68642BE8
:107534000ED90025104B0F4912481D702570FFF716
:10754400B1FD2946BDE8704064220E4800F049BCF4
:1075540070BD00BFE0040020DE040020040600200B
:10756400DC0400200C04002014040020E2040020A9
:10757400E1040020DF040020DD04002010040020CA
:107584007804002046050020AA05002003232DE9E5
:10759400F0410425BE27DFF8EC8086B08DF8093071
:1075A400344C98F8003029468DF80B3023780DF1CF
:1075B40009008DF80C308DF808708DF80A5000F031
:1075C40040FAEB261A2302218DF80D000DF101007B
:1075D4008DF801308DF802108DF80E608DF8007072
:1075E40000F02FFA01238DF8113098F800308DF84F
:1075F40003008DF81330237829460DF111008DF81E
:1076040014308DF804608DF810708DF8125000F06D
:1076140018FA194B8DF815001A788DF81660012A9E
:1076240026D1207820B9154A10605060144A107091
:107634000130C0B2082820708DF80C000FD9002545
:1076440028461D70FFF762FD9DF80210684603315D
:10765400C9B22570FFF714FD06B0BDE8F081FFF74D
:1076640055FD6420FCF724FE02A8FFF76BF8F3E74E
:1076740004A8FAE70A04002009040020AF0300204C
:10768400AE0300200804002010B5094C2368B3F5AC
:10769400FA7F0BD94FF400410648FDF742F9002365
:1076A4004AF6AA222360044B1B681A6010BD00BF6F
:1076B400FC0300200010014008060020054B5B6A13
:1076C4009B0005D50122044B04481A6000F01ABC43
:1076D400704700BF00100240E0044242519100088C
:1076E40010B590B02822002106A800F07AFB0021F2
:1076F400142201A800F075FB092301220693022439
:107704004FF4803306A807930A920C920E930D94BB
:10771400FDF73AFD0F23002101934FF4806301A884
:107724000294039104930591FDF7F6FE10B010BD89
:10773400BE232DE980488DB002268DF81830192318
:1077440031460DEB03004FF010098DF819308DF818
:107754001A6000F076F9EB23A24D8DF81C308DF8F9
:107764001B00FCF781FDFFF7BBFF4A46002108A878
:1077740000F037FBAB69002243EA0903AB61AB6954
:1077840049F6F07103EA09030293029BAB69964838
:1077940043F02003AB61AB69002403F0200303939F
:1077A400039BAB69012743F00403AB61AB69DFF8CA
:1077B400888203F004030493049BAB694FF00C0A22
:1077C40043F00803AB61AB694FF4E13B03F00803FA
:1077D4000593059BFDF7A0F8002248F2F0118348B9
:1077E400FDF79AF800224FF2E9318148FDF794F849
:1077F400002204217F48FDF78FF849F6F07308A9A9
:10780400794808930B9609970A94FCF793FF7A4BEF
:1078140008A97548099308970A94FCF78BFF48F266
:10782400F01308A9714808930B9609970A94FCF77A
:1078340081FF4FF2E93308A96D4808930B96099725
:107844000A94FCF777FF042308A96A4808930B9667
:1078540009970A94FCF76EFF08A96548CDF82090B3
:1078640009940A94FCF766FF6B69644A3B436B61B5
:107874006B6940463B400193019B40F23F6388E8BB
:107884000C0009235E4EC8F80C3008940994C8F81B
:107894000840C8F81840FEF70FF808A940460894B5
:1078A4000994FEF723F8574B574D304686E80808ED
:1078B400C6F814A0B460F4603461B461F461FEF7F6
:1078C4000DF9524B284685E80808C5F814A0AC60A9
:1078D400EC602C61AC61EC61FEF700F94C484D4959
:1078E4004D4BDFF858A180E80A004FF480438460D0
:1078F4000361C46044618461C4610462FDF7ECF90E
:10790400464B50468AE818004FF47A73CAF8083098
:10791400FDF718FC224621460F20FCF7EDFC0F2052
:10792400FCF71EFD224621462520FCF7E5FC252018
:10793400FCF716FD224621462620FCF7DDFC262016
:10794400FCF70EFD224621463620FCF7D5FC3620F6
:10795400FCF706FD224621464846FCF7CDFC484686
:10796400FCF7FEFC224621460620FCF7C5FC062057
:10797400FCF7F6FC4046FDF7A1FE294B3A4629499F
:1079840030461F70FEF734F93A4627492846FEF779
:107994002FF9264B21461B68254D986800F0BAFA4A
:1079A4009DF81A1006A80331C9B2FFF769FBFFF767
:1079B40085FE4CF6CC42DAF800301E4E1A60FEF713
:1079C4004FFBFFF7B5FC2B68B34288BF2C60FEF772
:1079D400A9FDFFF7E9FCFFF759FDFFF7D7FDFFF716
:1079E40053FEF0E70010024000100140000801407F
:1079F400000C014000140140000011100010004070
:107A04003407002000380140E00800200044004012
:107A14001406002000580040A086010000300040F9
:107A2400090400203C0800206806002014000020FF
:107A340004040020E0930400A008002008060020AD
:107A4400704710B5FF230446221AD2B2914201D8DE
:107A5400184610BD14F8012B5340082213F0800F70
:107A640002F1FF324FEA430318BF83F0310312F0EF
:107A7400FF02DBB2F2D1E7E730B5FF2305462C1A4B
:107A8400E4B2A14203D89B1A5842584130BD15F8BC
:107A9400014B6340082413F0800F04F1FF344FEAD4
:107AA400430318BF83F0310314F0FF04DBB2F2D1B7
:107AB400E5E700000E4B82B09A6942F001029A6138
:107AC4009A6902F001020092009ADA6942F0805247
:107AD400DA61DB69074A03F080530193019B536821
:107AE40023F0E06343F08063536002B0704700BF4B
:107AF400001002400000014010B5044686B0102278
:107B0400002102A800F06DF92268114B9A421DD1A0
:107B1400104C02A9A369104843F00803A361A369A8
:107B240003F008030093009B4FF440630293122375
:107B3400039303230593FCF7FDFDE36943F48003FA
:107B4400E361E36903F480030193019B06B010BD74
:107B54000058004000100240000C01400268084B2D
:107B640082B09A420AD103F50033DA6942F0100276
:107B7400DA61DB6903F010030193019B02B07047E3
:107B840000100040102270B5064688B00DEB0200CC
:107B9400002100F026F93368364A93423DD1364B32
:107BA40004A99A69354842F480429A619A69002589
:107BB40002F480420092009A9A69314C42F0040225
:107BC4009A619B6903F004030193019B4FF40073D2
:107BD40004930223059303230793FCF7ABFD4FF4AF
:107BE400806304A92548049305950695FCF7A2FD36
:107BF400244B84E828008023E3602023A5602561CA
:107C04006561A361E5612046FCF7CCFB08B1FFF791
:107C140017FF7463666208B070BD1B4A9342FAD1C1
:107C2400154B04A9DA69154842F40032DA61DA69BD
:107C3400002502F400320292029A9A69134C42F02F
:107C440004029A619B6903F004030393039B0423D6
:107C540004930223059303230793FCF76BFD082386
:107C640004A90648049305950695FCF763FD084BA3
:107C7400BFE700BF00380140001002400008014087
:107C8400F00600205800024000440040BC050020DB
:107C94006C0002407047FEE7FEE7FEE7FEE7704730
:107CA40070477047FCF7F2BA0120FCF73FBE0000B2
:107CB4000148FCF763BC00BFF00600200148FCF754
:107CC4005DBC00BFBC0500200148FEF763B800BFDF
:107CD400340700200148FEF75DB800BFE00800202B
:107CE4000148FDF7FABC00BFA00800200E4B1A683B
:107CF40042F001021A6059680C4A0A405A601A6834
:107D040022F0847222F480321A601A6822F48022EB
:107D14001A605A6822F4FE025A604FF41F029A60F5
:107D2400034A044B9A607047001002400000FFF8B9
:107D34000040000800ED00E0002103E00B4B5B581D
:107D4400435004310A480B4B42189A42F6D30A4A6C
:107D540002E0002342F8043B084B9A42F9D3FFF7B0
:107D6400C5FF00F00FF8FFF7E3FC7047209200080E
:107D74000000002078000020780000203C0A002049
:107D8400FEE7000070B500250C4E0D4CA41BA4109A
:107D9400A54209D101F0D4F800250A4E0A4CA41BCF
:107DA400A410A54205D170BD56F825309847013579
:107DB400EEE756F8253098470135F2E718920008A7
:107DC40018920008189200081C92000810B5431E6F
:107DD4000A44914200D110BD11F8014B03F8014F40
:107DE400F7E703460244934200D1704703F8011BAE
:107DF400F9E700000FB40A4B13B51C6824B1A3695A
:107E040013B9204600F0EEFA05AB049AA1682046A7
:107E1400019300F0AFFC02B0BDE8104004B070471D
:107E24001400002038B5084B05461C6824B1A3692A
:107E340013B9204600F0D6FAA26829462046BDE8C8
:107E4400384000F045BF00BF1400002070B50E4656
:107E5400054618B183690BB900F0C4FAAB69AC6884
:107E640013B9284600F0BEFA234B9C4217D16C6824
:107E7400A3891B071DD52369DBB1013EA36816F84E
:107E8400011F013BA360E9B9002B2EDA22460A2127
:107E9400284600F0F5F8013011D00A2070BD174BC8
:107EA4009C4201D1AC68E3E7154B9C4208BFEC68E7
:107EB400DEE72146284600F035F90028DDD04FF0F2
:107EC400FF3070BD002B04DAA269934206DB0A2955
:107ED40004D023685A1C22601970CFE72246284632
:107EE40000F0CEF80130C9D1E9E70A2023685A1C12
:107EF4002260187070BD00BFA4910008C4910008EE
:107F040084910008024B01461868FFF79FBF00BF29
:107F14001400002000294FF480630CBF02220022C9
:107F240000F000B82DE9F7431D46514B04461E6886
:107F34000F46904626B1B36913B9304600F052FAA1
:107F44004C4B9C4252D17468B8F1020F06D0B8F180
:107F5400010F00F28980002DC0F286802146304650
:107F640000F0D6F9616B41B104F14403994202D0A7
:107F7400304600F02DFB002363630023A36163609C
:107F8400A3891B0603D52169304600F021FBA38990
:107F9400B8F1020F23F44A6323F00303A3815DD0F5
:107FA40001AB6A462146304600F0A6FAA38918437D
:107FB400A0812DBB009D284600F002FB0746002847
:107FC4004ED1DDF80090A9453CD14FF0FF30A38994
:107FD40043F00203A3810023A36004F14703236059
:107FE40023610123636103B0BDE8F083224B9C420B
:107FF40001D1B468A8E7214B9C4208BFF468A3E709
:10800400002FD8D0B36913B9304600F0EBF9B8F1BA
:10801400010F08BFA389276004BF43F00103A381B4
:10802400A389276113F0080065611BD013F00100D8
:108034004FF000031FBF6D42A360A561184608BF3F
:10804400A560D0E7484600F0BBFA07460028BCD03C
:10805400A3894D4643F08003A381D3E70020B6E70C
:10806400A946F5E7A060BEE74FF0FF30BBE700BFCD
:1080740014000020A4910008C49100088491000811
:10808400F8B50E461446054618B183690BB900F0DD
:10809400A9F9214B9C422AD16C68A369A360A389E6
:1080A4001A072ED5236963B323692068F6B2C01A70
:1080B40063693746984204DB2146284600F028F9D4
:1080C40028BBA3680130013BA36023685A1C2260CB
:1080D4001E706369984204D0A389DB0719D50A2E60
:1080E40017D12146284600F013F990B10FE00B4B4D
:1080F4009C4201D1AC68D0E7094B9C4208BFEC68B4
:10810400CBE72146284600F00DF80028CCD04FF0EC
:10811400FF373846F8BD00BFA4910008C491000899
:1081240084910008324B70B51D6806460C4625B193
:10813400AB6913B9284600F055F92E4B9C420FD178
:108144006C68B4F90C309AB215072CD4D00611D44B
:108154000922326043F04003A3814FF0FF3070BD29
:10816400254B9C4201D1AC68EBE7244B9C4208BFF1
:10817400EC68E6E7510712D5616B41B104F14403A1
:10818400994202D0304600F023FA00236363A389A6
:1081940023F02403A3810023636023692360A3895C
:1081A40043F00803A38123694BB9A38903F4207323
:1081B400B3F5007F03D02146304600F0C1F9A2890F
:1081C40012F001030CD00023A36063695B42A36136
:1081D400236953B9B4F90C3013F08000BAD170BDDF
:1081E400920758BF6369A360F2E70020F7E700BF76
:1081F40014000020A4910008C49100088491000890
:108204008A892DE9F041054610070C465AD44B687B
:10821400002B05DC0B6C002B02DC0020BDE8F08198
:10822400E66A002EF9D0002312F480522F682B60E6
:1082340033D0606DA3895A0705D56368C01A636B90
:108244000BB1236CC01A00230246E66A216A284651
:10825400B047431CA38906D129681D294BD82B4A52
:10826400CA40D60747D5002262602269D904226039
:1082740004D5421C01D12B6803B96065616B2F6082
:108284000029CAD004F14403994202D0284600F0E0
:108294009FF900206063BDE8F081216A012328462C
:1082A400B047411CC6D12B68002BC3D01D2B01D075
:1082B400162B01D12F60B0E7A38943F04003A381BB
:1082C400BDE8F0810F69002FA7D0930718BF0023E2
:1082D4000E6808BF4B69A6EB07080F608B60B8F106
:1082E400000F9ADD43463A46216A2846A66AB047FB
:1082F400002807DCA38943F04003A3814FF0FF303B
:10830400BDE8F0810744A8EB0008E8E7010040203D
:1083140038B50B6905460C46DBB118B183690BB956
:1083240000F060F80C4B9C4209D16C68B4F90C3035
:108334007BB121462846BDE83840FFF761BF074BB3
:108344009C4201D1AC68F1E7054B9C4208BFEC6844
:10835400ECE7002038BD00BFA4910008C4910008D8
:1083640084910008014900F0A9B800BF15830008F2
:10837400002310B504460360436083608181436633
:10838400C281036143618361194608225C30FFF7AF
:1083940028FD054B24626362044BA362044BE36231
:1083A400044B236310BD00BF618D0008838D00085A
:1083B400BB8D0008DF8D000870B568254A1E554343
:1083C4000E4605F1740100F04FF9044640B1002156
:1083D40080E842000C30A06005F16802FFF701FD5F
:1083E400204670BD836910B5044633BB8364C364FF
:1083F4000365124B124A1B688262984204BF012330
:10840400836100F01FF86060204600F01BF8A06054
:10841400204600F017F80022E06004216068FFF7AE
:10842400A7FF01220921A068FFF7A2FF022212215F
:10843400E068FFF79DFF0123A36110BD8091000850
:1084440069830008F8B51C4B07461E68B36913B965
:108454003046FFF7C7FF4836B4687368013B03D55D
:10846400336833B13668F7E7B4F90C506DB168344A
:10847400F4E704213846FFF79FFF30600028F1D16C
:108484000C2304463B602046F8BD4FF6FF73E3819E
:1084940001236566A3812560A5606560256165612A
:1084A400A5610822294604F15C00FFF79AFC656384
:1084B400A563A564E564E6E7809100082DE9F84327
:1084C40080468946002600F1480414B93046BDE8C8
:1084D400F883A5686768013F01D52468F5E7AB898F
:1084E400012B07D9B5F90E30013303D02946404694
:1084F400C84706436835EEE770B50E46B1F90E106D
:1085040090B0002914461D4607DA00232B60B38976
:108514001A0610D44FF480630EE001AA00F084FC24
:108524000028F2DB029A02F47042A2F500535A4288
:108534005A412A60EEE740230020236010B070BD4A
:108544008B8973B59D0706460C4607D504F147038E
:10855400236023610123636102B070BD01AB6A46ED
:10856400FFF7CAFF00990546304600F07DF848B988
:10857400B4F90C309A05EFD423F0030343F002035B
:10858400A381E3E70D4BB362A389206043F080032A
:10859400A381009B20616361019B5BB1B4F90E1060
:1085A400304600F053FC28B1A38923F0030343F0C1
:1085B4000103A381A3891D43A581CDE76983000835
:1085C400024B0146186800F04FB800BF14000020A9
:1085D40038B50546002943D051F8043C0C1F002B44
:1085E400B8BFE41800F062FC1E4A1368104633B9A1
:1085F400636014602846BDE8384000F058BCA342CC
:108604000BD921686218934201BF1A685B6852183B
:10861400226063600460EDE713465A680AB1A2421F
:10862400FAD919685818A0420BD120680144581887
:1086340082421960DED110685268014419605A60A0
:10864400D8E702D90C232B60D4E7206821188A428A
:1086540001BF116852680918216062605C60C9E753
:1086640038BD00BFAC05002070B5CD1C25F0030556
:1086740008350C2D38BF0C25002D064601DBA94218
:1086840003D90C233360002070BD00F00FFC234A93
:108694001468214691B9224C23681BB9304600F076
:1086A4004DFB20602946304600F048FB431C26D190
:1086B4000C233046336000F0FAFBE4E70B685B1BE5
:1086C4001AD40B2B0FD90B60CC18CD50304600F0C8
:1086D400EEFB04F10B00231D20F00700C31A1BD08E
:1086E4005A42E25070BD8C420BBF63684B68136002
:1086F400636018BF0C46E9E70C464968CAE7C41C26
:1087040024F00304A04205D0211A304600F016FBE1
:108714000130CDD02560D9E770BD00BFAC05002085
:10872400B0050020936810B4013B002B936008DA75
:108734009469A34202DBCBB20A2B02D110BCFFF72F
:108744009FBC1368581C10601970C8B210BC7047E5
:10875400F8B506460F461446D518AC4201D10020A0
:1087640007E03A4614F8011B3046FFF7DBFF431CD1
:10877400F3D1F8BD2DE9F04F9DB00C461746039395
:10878400064618B183690BB9FFF72CFE7C4B9C425B
:1087940057D17468A38918075DD52369002B5AD073
:1087A4000023099320238DF8293030234FF0010B47
:1087B4008DF82A30B846454615F8013B002B55D1B3
:1087C400B8EB070A0BD053463A4621463046FFF72A
:1087D400BFFF013000F0C480099B5344099398F80B
:1087E4000030002B00F0BC8000234FF0FF320493D4
:1087F4000793059206938DF853301A93052229782E
:10880400604800F045FB05F10108049B002831D1C4
:10881400D90644BF20228DF853201A0744BF2B22C7
:108824008DF853202A782A2A2CD000210A20079A6E
:10883400A84698F800300135303B092B6DD971B347
:1088440026E0514B9C4201D1B468A3E74F4B9C42B4
:1088540008BFF4689EE721463046FFF763FC002812
:108864009ED04FF0FF301DB0BDE8F08F252BA7D070
:10887400A846A0E7434A4546801A0BFA00F018437D
:108884000490BBE7039A111D12680391002A01DBCF
:10889400079204E0524243F002030792049398F8CB
:1088A40000302E2B10D198F8013008F101012A2B49
:1088B40037D1039B08F102081A1D1B680392002B91
:1088C400B8BF4FF0FF330593314D032298F80010E1
:1088D400284600F0DDFA40B14023401B03FA00F0C3
:1088E400049B08F101080343049398F8001006223E
:1088F400284808F101078DF8281000F0C9FA00286B
:1089040034D0254B03BB039B073323F00703083301
:108914000393099B4B4409934CE700FB023201216A
:1089240086E700230A2518460593884698F8002010
:108934000131303A092A03D9002BC5D00590C3E789
:1089440005FB00200123F0E703AB00932246134B01
:1089540004A93046AFF30080B0F1FF3F8146D8D17F
:10896400A3895B063FF57DAF09987CE703AB0093D1
:1089740022460A4B04A9304600F08AF8ECE700BF0F
:10898400A4910008E4910008C491000884910008AF
:10899400EA910008EE9100080000000055870008E5
:1089A4002DE9F04791461F468A680B6906469342B3
:1089B400B8BF1346C9F8003091F843200C46DDF8DF
:1089C400208012B10133C9F800302368990642BFF0
:1089D400D9F800300233C9F80030256815F00605CF
:1089E40007D104F1190AE368D9F800209B1A9D42C3
:1089F4002ADB94F843302268003318BF012392061F
:108A04002FD404F1430239463046C047013022D006
:108A14002368E56803F00603042B18BF0025D9F882
:108A240000204FF0000908BFAD1AA368226908BFEF
:108A340025EAE5759342C4BF9B1AED181A344D45D7
:108A44001BD10020BDE8F087012352463946304649
:108A5400C047013003D14FF0FF30BDE8F087013546
:108A6400C1E73020E11881F843005A1C94F84510FE
:108A74002244023382F84310C3E7012322463946D5
:108A84003046C0470130E6D009F10109D7E70000BC
:108A94002DE9F04317460A7E85B06E2A98460646AD
:108AA4000C460C9B01F1430E00F0BC801AD8632ADB
:108AB4002ED00AD8002A00F0C880582A00F08A80F4
:108AC40004F1420584F842202AE0642A01D0692A8C
:108AD400F6D121681A6811F0800F23D0111D196096
:108AE400136827E0732A00F0B48008D86F2A2AD0CC
:108AF400702AE5D10A6842F020020A6003E0752A70
:108B040021D0782ADCD178226F4984F8452064E0AA
:108B14001A6801F14205111D1960136884F8423086
:108B24000123A3E011F0400F02F104011960D7D032
:108B3400B2F90030002B03DA2D225B4284F8432083
:108B440062490A2217E02068196810F0800F03D0E8
:108B5400081D18600B6806E010F0400F01F10400D6
:108B64001860F7D00B886F2A14BF0A2208225749CD
:108B7400002084F843006568002DA560C0F29C8045
:108B8400206820F004002060002B3FD1002D40F02D
:108B940095807546082A0BD12368DA0708D523691E
:108BA40062689A42DEBF302305F8013C05F1FF35C7
:108BB400AEEB05032361CDF800803B4603AA2146B2
:108BC4003046FFF7EDFE013055D14FF0FF3005B0D0
:108BD400BDE8F08381F845203C492268186812F00A
:108BE400800F00F104051D6001D0036802E0550602
:108BF400FBD50388D00744BF42F0200222601BB992
:108C0400226822F0200222601022B1E77546B3FBED
:108C1400F2F002FB1033CB5C05F8013D034600285B
:108C2400F5D1B7E708681A6810F0800F496904D0D5
:108C3400101D18601368196007E010F0400F02F16E
:108C4400040018601368F6D0198000237546236168
:108C5400B1E71A68111D1960156800216268284679
:108C640000F016F908B1401B6060636823610023BB
:108C740084F843309FE723692A4639463046C04783
:108C84000130A2D023689B0707D5002504F11909F8
:108C9400E368039A9B1A9D4205DBE068039B9842B4
:108CA400B8BF184693E701234A4639463046C047C1
:108CB40001308AD00135EBE7002BA7D10B7804F102
:108CC400420584F8423065E706920008F5910008F1
:108CD40070B50D461446064618B183690BB9FFF703
:108CE40081FB134B9C4212D17468A368013B002B97
:108CF400A36016DAA269934202DBEBB20A2B10D10D
:108D0400224629463046BDE87040FFF7B9B9094B01
:108D14009C4201D1B468E8E7074B9C4208BFF46861
:108D2400E3E72368E8B25A1C22601D7070BD00BFDF
:108D3400A4910008C49100088491000838B5002368
:108D4400054C05460846236000F0ECF8431C02D1AC
:108D5400236803B12B6038BD380A002010B50C46D7
:108D6400B1F90E1000F0A4F80028ABBF636DA3891D
:108D74001B1823F48053ACBF6365A38110BD2DE998
:108D8400F0411F468B890546DB050C46164605D582
:108D940002230022B1F90E1000F068F8A3893246CC
:108DA40023F48053A381B4F90E103B462846BDE852
:108DB400F04100F017B810B50C46B1F90E1000F0F0
:108DC40055F8431CA38915BF606523F4805343F40D
:108DD4008053A38118BFA38110BDB1F90E1000F018
:108DE40013B8000038B50546084611460022054C64
:108DF40022601A46FEF74CF9431C02D1236803B1E2
:108E04002B6038BD380A002038B50023054C0546D0
:108E14000846236000F05EF8431C02D1236803B1C6
:108E24002B6038BD380A002038B50023064C0546AF
:108E340008461146236000F055F8431C02D123680C
:108E440003B12B6038BD00BF380A002038B50023B9
:108E5400054C05460846236000F04CF8431C02D13B
:108E6400236803B12B6038BD380A002038B50546A5
:108E7400084611460022054C22601A4600F042F8CA
:108E8400431C02D1236803B12B6038BD380A00208B
:108E940010B5C9B202449042034601D1002010BD6E
:108EA4001C7801308C42F6D1184610BD70477047CB
:108EB40038B50546084611460022054C22601A467C
:108EC40000F028F8431C02D1236803B12B6038BD9D
:108ED400380A00205822024B4FF0FF301A607047C6
:108EE400380A00205822024B4FF0FF301A607047B6
:108EF400380A00205822024B00201A60704700BF35
:108F0400380A00205822024B4FF0FF301A60704795
:108F1400380A00205822024B4FF0FF301A60704785
:108F2400380A0020044B0246196809B9034919603C
:108F3400186802441A607047B40500203C0A0020F7
:108F4400F8B500BFF8BC08BC9E467047F8B500BF32
:088F5400F8BC08BC9E46704702
:108F5C0002030405060708090A0B0C0D0E0F10106E
:108F6C00454550524F4D2053415645204552524F86
:108F7C0052212121200001070D13191F252B32002E
:108F8C0064009600C800FA002C015E0190010407F1
:108F9C000A0D101D20235265636F676E697A652078
:108FAC0025642053656E736F720A004D59206964F5
:108FBC00206973202564200A005247425F53656E76
:108FCC00736F725265644C696D69745F4275665B50
:108FDC0025645D202020203A2020253034780A009A
:108FEC005247425F53656E736F72477265656E4C84
:108FFC00696D69745F4275665B25645D20203A205B
:10900C0020253034780A005247425F53656E736FE7
:10901C0072426C75654C696D69745F4275665B254F
:10902C00645D2020203A2020253034780A004C6FD3
:10903C007261206672657175656E6379203A2025C0
:10904C0064200A004C6F726120706F77657220206B
:10905C002020203A202564200A004C6F7261204C9D
:10906C006F52615F52617465203A202564200A00BA
:10907C004C6F7261204C6F52615F42572020203A36
:10908C00202564200A004C6F7261204C6F52615F86
:10909C004C6E6120203A202564200A004E6F74200B
:1090AC004578697374204465766963652000E540F2
:1090BC0026E56026E58026E5A026E5C026E5E02627
:1090CC00E60026E62026E64026E66026E68026E632
:1090DC00A026E6C026E6E0260001020304050607EA
:1090EC000809FFFCF9F6060708090A0B0C5478204E
:1090FC00627566666572203A200052656365697612
:10910C0065642044617461203A2000253032782057
:10911C00004F726967696E616C20435243203A209C
:10912C00253032782052656376435243203A20250D
:10913C00303278200D0A00576861742048617070D5
:10914C00656E3F0D004920616D205265736574207A
:10915C00466C616720436C65617200000000000082
:10916C0000000001020304060708090000000001CA
:10917C0002030400180000200000000000000000A2
:10918C0000000000000000000000000000000000D3
:10919C0000000000000000000000000000000000C3
:1091AC0000000000000000000000000000000000B3
:1091BC0000000000000000000000000000000000A3
:1091CC000000000000000000000000000000000093
:1091DC000000000000000000232D302B2000686CE4
:1091EC004C006566674546470030313233343536BE
:1091FC0037383941424344454600303132333435F7
:0C920C0036373839616263646566000023
:0492180009420008FF
:04921C00E541000820
:109220000100000010000000000102030A0100001C
:1092300000A24A041800002000000000A4910008C9
:10924000C4910008849100080000000000000000A4
:10925000000000000000000000000000000000000E
:1092600000000000000000000000000000000000FE
:1092700000000000000000000000000000000000EE
:1092800000000000000000000000000000000000DE
:089290000000000000000000D6
:0400000508007D3D35
:00000001FF
